Archive member included because of file (symbol)

c:/winavr-20100110/bin/../lib/gcc/avr/4.3.3/avr4\libgcc.a(_udivmodhi4.o)
                              main.o (__udivmodhi4)
c:/winavr-20100110/bin/../lib/gcc/avr/4.3.3/avr4\libgcc.a(_exit.o)
                              c:/winavr-20100110/bin/../lib/gcc/avr/4.3.3/../../../../avr/lib/avr4/crtm88.o (exit)
c:/winavr-20100110/bin/../lib/gcc/avr/4.3.3/avr4\libgcc.a(_copy_data.o)
                              cc1100.o (__do_copy_data)
c:/winavr-20100110/bin/../lib/gcc/avr/4.3.3/avr4\libgcc.a(_clear_bss.o)
                              cc1100.o (__do_clear_bss)
c:/winavr-20100110/bin/../lib/gcc/avr/4.3.3/../../../../avr/lib/avr4\libc.a(strtok.o)
                              main.o (strtok)
c:/winavr-20100110/bin/../lib/gcc/avr/4.3.3/../../../../avr/lib/avr4\libc.a(memcmp.o)
                              main.o (memcmp)
c:/winavr-20100110/bin/../lib/gcc/avr/4.3.3/../../../../avr/lib/avr4\libc.a(memset.o)
                              main.o (memset)
c:/winavr-20100110/bin/../lib/gcc/avr/4.3.3/../../../../avr/lib/avr4\libc.a(strcpy.o)
                              main.o (strcpy)
c:/winavr-20100110/bin/../lib/gcc/avr/4.3.3/../../../../avr/lib/avr4\libc.a(strstr.o)
                              main.o (strstr)
c:/winavr-20100110/bin/../lib/gcc/avr/4.3.3/../../../../avr/lib/avr4\libc.a(strtok_r.o)
                              c:/winavr-20100110/bin/../lib/gcc/avr/4.3.3/../../../../avr/lib/avr4\libc.a(strtok.o) (strtok_r)
c:/winavr-20100110/bin/../lib/gcc/avr/4.3.3/../../../../avr/lib/avr4\libc.a(eerd_block_atmega88.o)
                              main.o (__eerd_block_m88)
c:/winavr-20100110/bin/../lib/gcc/avr/4.3.3/../../../../avr/lib/avr4\libc.a(eerd_byte_atmega88.o)
                              main.o (__eerd_byte_m88)
c:/winavr-20100110/bin/../lib/gcc/avr/4.3.3/../../../../avr/lib/avr4\libc.a(eewr_block_atmega88.o)
                              main.o (__eewr_block_m88)
c:/winavr-20100110/bin/../lib/gcc/avr/4.3.3/../../../../avr/lib/avr4\libc.a(eewr_byte_atmega88.o)
                              c:/winavr-20100110/bin/../lib/gcc/avr/4.3.3/../../../../avr/lib/avr4\libc.a(eewr_block_atmega88.o) (__eewr_r18_m88)

Allocating common symbols
Common symbol       size              file

uart_rx_length      0x1               main.o
uart_data           0x1               main.o
gTestMode           0x1               main.o
SRBufIndex          0x1               main.o
gOpt                0xf               main.o
tSlave              0x4               main.o
pC                  0x2               main.o
gClient             0x49              main.o
gLevel              0x1               main.o
gggLength           0x1               main.o
tSlave2             0x4               main.o
gTemperature        0x2               main.o
SRBuf               0x4               main.o
gWCmd               0x60              main.o
tCtl                0x7               main.o
rx_char             0x3c              main.o
cmd                 0x28              main.o

Memory Configuration

Name             Origin             Length             Attributes
text             0x00000000         0x00002000         xr
data             0x00800060         0x0000ffa0         rw !x
eeprom           0x00810000         0x00010000         rw !x
fuse             0x00820000         0x00000400         rw !x
lock             0x00830000         0x00000400         rw !x
signature        0x00840000         0x00000400         rw !x
*default*        0x00000000         0xffffffff

Linker script and memory map

Address of section .data set to 0x800100
LOAD c:/winavr-20100110/bin/../lib/gcc/avr/4.3.3/../../../../avr/lib/avr4/crtm88.o
LOAD cc1100.o
LOAD main.o
LOAD spi1.o
LOAD i2c.o
LOAD c:/winavr-20100110/bin/../lib/gcc/avr/4.3.3/avr4\libgcc.a
LOAD c:/winavr-20100110/bin/../lib/gcc/avr/4.3.3/../../../../avr/lib/avr4\libc.a
LOAD c:/winavr-20100110/bin/../lib/gcc/avr/4.3.3/avr4\libgcc.a

.hash
 *(.hash)

.dynsym
 *(.dynsym)

.dynstr
 *(.dynstr)

.gnu.version
 *(.gnu.version)

.gnu.version_d
 *(.gnu.version_d)

.gnu.version_r
 *(.gnu.version_r)

.rel.init
 *(.rel.init)

.rela.init
 *(.rela.init)

.rel.text
 *(.rel.text)
 *(.rel.text.*)
 *(.rel.gnu.linkonce.t*)

.rela.text
 *(.rela.text)
 *(.rela.text.*)
 *(.rela.gnu.linkonce.t*)

.rel.fini
 *(.rel.fini)

.rela.fini
 *(.rela.fini)

.rel.rodata
 *(.rel.rodata)
 *(.rel.rodata.*)
 *(.rel.gnu.linkonce.r*)

.rela.rodata
 *(.rela.rodata)
 *(.rela.rodata.*)
 *(.rela.gnu.linkonce.r*)

.rel.data
 *(.rel.data)
 *(.rel.data.*)
 *(.rel.gnu.linkonce.d*)

.rela.data
 *(.rela.data)
 *(.rela.data.*)
 *(.rela.gnu.linkonce.d*)

.rel.ctors
 *(.rel.ctors)

.rela.ctors
 *(.rela.ctors)

.rel.dtors
 *(.rel.dtors)

.rela.dtors
 *(.rela.dtors)

.rel.got
 *(.rel.got)

.rela.got
 *(.rela.got)

.rel.bss
 *(.rel.bss)

.rela.bss
 *(.rela.bss)

.rel.plt
 *(.rel.plt)

.rela.plt
 *(.rela.plt)

.text           0x00000000     0x1db2
 *(.vectors)
 .vectors       0x00000000       0x34 c:/winavr-20100110/bin/../lib/gcc/avr/4.3.3/../../../../avr/lib/avr4/crtm88.o
                0x00000000                __vectors
                0x00000000                __vector_default
 *(.vectors)
 *(.progmem.gcc*)
 *(.progmem*)
                0x00000034                . = ALIGN (0x2)
                0x00000034                __trampolines_start = .
 *(.trampolines)
 .trampolines   0x00000034        0x0 linker stubs
 *(.trampolines*)
                0x00000034                __trampolines_end = .
 *(.jumptables)
 *(.jumptables*)
 *(.lowtext)
 *(.lowtext*)
                0x00000034                __ctors_start = .
 *(.ctors)
                0x00000034                __ctors_end = .
                0x00000034                __dtors_start = .
 *(.dtors)
                0x00000034                __dtors_end = .
 SORT(*)(.ctors)
 SORT(*)(.dtors)
 *(.init0)
 .init0         0x00000034        0x0 c:/winavr-20100110/bin/../lib/gcc/avr/4.3.3/../../../../avr/lib/avr4/crtm88.o
                0x00000034                __init
 *(.init0)
 *(.init1)
 *(.init1)
 *(.init2)
 .init2         0x00000034        0xc c:/winavr-20100110/bin/../lib/gcc/avr/4.3.3/../../../../avr/lib/avr4/crtm88.o
 *(.init2)
 *(.init3)
 *(.init3)
 *(.init4)
 .init4         0x00000040       0x16 c:/winavr-20100110/bin/../lib/gcc/avr/4.3.3/avr4\libgcc.a(_copy_data.o)
                0x00000040                __do_copy_data
 .init4         0x00000056       0x10 c:/winavr-20100110/bin/../lib/gcc/avr/4.3.3/avr4\libgcc.a(_clear_bss.o)
                0x00000056                __do_clear_bss
 *(.init4)
 *(.init5)
 *(.init5)
 *(.init6)
 *(.init6)
 *(.init7)
 *(.init7)
 *(.init8)
 *(.init8)
 *(.init9)
 .init9         0x00000066        0x4 c:/winavr-20100110/bin/../lib/gcc/avr/4.3.3/../../../../avr/lib/avr4/crtm88.o
 *(.init9)
 *(.text)
 .text          0x0000006a        0x2 c:/winavr-20100110/bin/../lib/gcc/avr/4.3.3/../../../../avr/lib/avr4/crtm88.o
                0x0000006a                __vector_22
                0x0000006a                __vector_24
                0x0000006a                __vector_12
                0x0000006a                __bad_interrupt
                0x0000006a                __vector_6
                0x0000006a                __vector_3
                0x0000006a                __vector_23
                0x0000006a                __vector_25
                0x0000006a                __vector_11
                0x0000006a                __vector_13
                0x0000006a                __vector_17
                0x0000006a                __vector_19
                0x0000006a                __vector_7
                0x0000006a                __vector_5
                0x0000006a                __vector_4
                0x0000006a                __vector_9
                0x0000006a                __vector_21
                0x0000006a                __vector_15
                0x0000006a                __vector_8
                0x0000006a                __vector_14
                0x0000006a                __vector_10
                0x0000006a                __vector_16
                0x0000006a                __vector_20
 .text          0x0000006c      0x20a cc1100.o
                0x0000015e                cc1100_strobe_cmd
                0x00000080                cc1100_sleep_strobe_cmd
                0x000001ec                cc1100_read_status
                0x00000076                cc1100_gdo2_register_callback
                0x00000132                cc1100_fifo_put
                0x000001f6                cc1100_init
                0x00000106                cc1100_fifo_get
                0x000000ae                cc1100_write_reg
                0x00000180                cc1100_cmd_idle
                0x000001f2                cc1100_reinit
                0x000000d0                cc1101_init_reg
                0x000001cc                cc1100_read_reg
                0x000001ba                cc1100_cmd_calibrate
                0x0000006c                cc1100_gdo0_register_callback
                0x00000084                cc1101_8PATABLE_write_reg
                0x000000ee                cc1101_rtx_reg_set
 .text          0x00000276     0x1796 main.o
                0x0000028c                mdelay
                0x00000550                get_input_data
                0x000009a0                sleep_set
                0x00000808                __vector_1
                0x000002fe                putb
                0x0000077c                insert_sr_buf
                0x00000d60                cc1101_carrier_wave_setup
                0x00000f88                cc1101_tx_carrier
                0x00000440                led_onoff
                0x0000036a                putstr
                0x00000346                chr2hex
                0x00000b12                tx_fifo_write
                0x000002ee                putc_
                0x0000178c                slave_oper
                0x00000320                puthex
                0x00000d58                my_eeprom_read_byte
                0x00000ca2                reg_slave_num_serch
                0x00001004                master_oper
                0x00000ab4                rx_fifo_read
                0x00000e90                random_tx_test
                0x00000478                inituart
                0x00001680                setup_oper
                0x000008a4                temperature_test_disenable
                0x000007f2                get_alarm_time
                0x000002c6                sdelay
                0x000008c4                temperature_get
                0x000015d0                slave_fifo_preset
                0x00000b42                my_eeprom_read_block
                0x0000041c                hexToAsc
                0x00000702                master_fifo_preset
                0x000005ce                get_frq
                0x000003e0                asc_to_int
                0x0000129e                master_main
                0x000006c0                sig_status
                0x00000618                sig_set
                0x00000c66                device_status_setup
                0x00000276                udelay
                0x00001766                setup_main
                0x00000334                putchr2hex
                0x0000040e                hex_to_asc
                0x00001806                slave_main
                0x00000398                asc_to_hex
                0x00000f0e                cc1101_tx
                0x00000ebe                cc1101_rx
                0x000003ea                AscToInt
                0x0000049a                hw_setup
                0x000008b2                temperature_test_enable
                0x000003bc                AscToHex
                0x00001960                main
                0x000004d6                ad_get_val
                0x00000b4a                check_env
                0x00000a1c                __vector_2
                0x000005f0                add_batt_low
                0x00000900                rtc_set_next_alarm
                0x000006fc                carrier_no_sense
                0x0000044c                led_flasher
                0x000009fe                rtc_alarm_disenable
                0x00000fdc                temperature_carrier_test
                0x00000864                hex_change_level
                0x0000058c                level_change_hex
                0x000005e4                init_voltcomparator
                0x000006f6                carrier_sense
                0x00000704                my_memcmp
                0x0000072a                __vector_18
                0x0000060e                get_sr_status
 .text          0x00001a0c       0xd6 spi1.o
                0x00001a6a                spi1_read
                0x00001aa0                spi1_read_somi
                0x00001a1e                spi1_write_single
                0x00001ac6                spi_signalpin_opendrain_nonactive
                0x00001a98                spi1_deselect
                0x00001a42                spi1_write
                0x00001aac                spi_signalpin_opendrain_active
                0x00001a30                spi1_read_single
                0x00001a0c                spi1_init
                0x00001a90                spi1_select
 .text          0x00001ae2      0x186 i2c.o
                0x00001b66                i2c_read_nak
                0x00001bf6                rtc_1byte_data_read
                0x00001b9a                i2c_write
                0x00001afe                i2c_wait_int_clear
                0x00001b80                i2c_read_ack
                0x00001b2a                i2c_start
                0x00001bb4                rtc_3byte_data_read
                0x00001aee                i2c_stop
                0x00001c26                rtc_1byte_data_write
                0x00001b1c                i2c_error
                0x00001ae2                i2c_init
 .text          0x00001c68        0x0 c:/winavr-20100110/bin/../lib/gcc/avr/4.3.3/avr4\libgcc.a(_udivmodhi4.o)
 .text          0x00001c68        0x0 c:/winavr-20100110/bin/../lib/gcc/avr/4.3.3/avr4\libgcc.a(_exit.o)
 .text          0x00001c68        0x0 c:/winavr-20100110/bin/../lib/gcc/avr/4.3.3/avr4\libgcc.a(_copy_data.o)
 .text          0x00001c68        0x0 c:/winavr-20100110/bin/../lib/gcc/avr/4.3.3/avr4\libgcc.a(_clear_bss.o)
 .text          0x00001c68        0x0 c:/winavr-20100110/bin/../lib/gcc/avr/4.3.3/../../../../avr/lib/avr4\libc.a(strtok.o)
 .text          0x00001c68        0x0 c:/winavr-20100110/bin/../lib/gcc/avr/4.3.3/../../../../avr/lib/avr4\libc.a(memcmp.o)
 .text          0x00001c68        0x0 c:/winavr-20100110/bin/../lib/gcc/avr/4.3.3/../../../../avr/lib/avr4\libc.a(memset.o)
 .text          0x00001c68        0x0 c:/winavr-20100110/bin/../lib/gcc/avr/4.3.3/../../../../avr/lib/avr4\libc.a(strcpy.o)
 .text          0x00001c68        0x0 c:/winavr-20100110/bin/../lib/gcc/avr/4.3.3/../../../../avr/lib/avr4\libc.a(strstr.o)
 .text          0x00001c68        0x0 c:/winavr-20100110/bin/../lib/gcc/avr/4.3.3/../../../../avr/lib/avr4\libc.a(strtok_r.o)
 .text          0x00001c68        0x0 c:/winavr-20100110/bin/../lib/gcc/avr/4.3.3/../../../../avr/lib/avr4\libc.a(eerd_block_atmega88.o)
 .text          0x00001c68        0x0 c:/winavr-20100110/bin/../lib/gcc/avr/4.3.3/../../../../avr/lib/avr4\libc.a(eerd_byte_atmega88.o)
 .text          0x00001c68        0x0 c:/winavr-20100110/bin/../lib/gcc/avr/4.3.3/../../../../avr/lib/avr4\libc.a(eewr_block_atmega88.o)
 .text          0x00001c68        0x0 c:/winavr-20100110/bin/../lib/gcc/avr/4.3.3/../../../../avr/lib/avr4\libc.a(eewr_byte_atmega88.o)
                0x00001c68                . = ALIGN (0x2)
 *(.text.*)
 .text.libgcc   0x00001c68       0x28 c:/winavr-20100110/bin/../lib/gcc/avr/4.3.3/avr4\libgcc.a(_udivmodhi4.o)
                0x00001c68                __udivmodhi4
 .text.libgcc   0x00001c90        0x0 c:/winavr-20100110/bin/../lib/gcc/avr/4.3.3/avr4\libgcc.a(_exit.o)
 .text.libgcc   0x00001c90        0x0 c:/winavr-20100110/bin/../lib/gcc/avr/4.3.3/avr4\libgcc.a(_copy_data.o)
 .text.libgcc   0x00001c90        0x0 c:/winavr-20100110/bin/../lib/gcc/avr/4.3.3/avr4\libgcc.a(_clear_bss.o)
 .text.avr-libc
                0x00001c90        0x8 c:/winavr-20100110/bin/../lib/gcc/avr/4.3.3/../../../../avr/lib/avr4\libc.a(strtok.o)
                0x00001c90                strtok
 .text.avr-libc
                0x00001c98       0x1a c:/winavr-20100110/bin/../lib/gcc/avr/4.3.3/../../../../avr/lib/avr4\libc.a(memcmp.o)
                0x00001c98                memcmp
 .text.avr-libc
                0x00001cb2        0xe c:/winavr-20100110/bin/../lib/gcc/avr/4.3.3/../../../../avr/lib/avr4\libc.a(memset.o)
                0x00001cb2                memset
 .text.avr-libc
                0x00001cc0        0xe c:/winavr-20100110/bin/../lib/gcc/avr/4.3.3/../../../../avr/lib/avr4\libc.a(strcpy.o)
                0x00001cc0                strcpy
 .text.avr-libc
                0x00001cce       0x34 c:/winavr-20100110/bin/../lib/gcc/avr/4.3.3/../../../../avr/lib/avr4\libc.a(strstr.o)
                0x00001cce                strstr
 .text.avr-libc
                0x00001d02       0x4e c:/winavr-20100110/bin/../lib/gcc/avr/4.3.3/../../../../avr/lib/avr4\libc.a(strtok_r.o)
                0x00001d02                strtok_r
 .text.avr-libc
                0x00001d50       0x20 c:/winavr-20100110/bin/../lib/gcc/avr/4.3.3/../../../../avr/lib/avr4\libc.a(eerd_block_atmega88.o)
                0x00001d54                __eerd_blraw_m88
                0x00001d50                __eerd_block_m88
 .text.avr-libc
                0x00001d70       0x10 c:/winavr-20100110/bin/../lib/gcc/avr/4.3.3/../../../../avr/lib/avr4\libc.a(eerd_byte_atmega88.o)
                0x00001d70                __eerd_byte_m88
 .text.avr-libc
                0x00001d80       0x12 c:/winavr-20100110/bin/../lib/gcc/avr/4.3.3/../../../../avr/lib/avr4\libc.a(eewr_block_atmega88.o)
                0x00001d80                __eewr_block_m88
 .text.avr-libc
                0x00001d92       0x1c c:/winavr-20100110/bin/../lib/gcc/avr/4.3.3/../../../../avr/lib/avr4\libc.a(eewr_byte_atmega88.o)
                0x00001d94                __eewr_r18_m88
                0x00001d92                __eewr_byte_m88
                0x00001dae                . = ALIGN (0x2)
 *(.fini9)
 .fini9         0x00001dae        0x0 c:/winavr-20100110/bin/../lib/gcc/avr/4.3.3/avr4\libgcc.a(_exit.o)
                0x00001dae                exit
                0x00001dae                _exit
 *(.fini9)
 *(.fini8)
 *(.fini8)
 *(.fini7)
 *(.fini7)
 *(.fini6)
 *(.fini6)
 *(.fini5)
 *(.fini5)
 *(.fini4)
 *(.fini4)
 *(.fini3)
 *(.fini3)
 *(.fini2)
 *(.fini2)
 *(.fini1)
 *(.fini1)
 *(.fini0)
 .fini0         0x00001dae        0x4 c:/winavr-20100110/bin/../lib/gcc/avr/4.3.3/avr4\libgcc.a(_exit.o)
 *(.fini0)
                0x00001db2                _etext = .

.data           0x00800100       0xb8 load address 0x00001db2
                0x00800100                PROVIDE (__data_start, .)
 *(.data)
 .data          0x00800100        0x0 c:/winavr-20100110/bin/../lib/gcc/avr/4.3.3/../../../../avr/lib/avr4/crtm88.o
 .data          0x00800100       0x1c cc1100.o
                0x00800100                pt_data
                0x00800108                init_all
 .data          0x0080011c       0x9b main.o
                0x00800166                reg_next_sch_alarm
                0x00800158                reg_net_alarm
                0x0080017f                level_offset
                0x00800178                day_cnt
                0x0080019b                default_offset
                0x0080017c                fix_id_mel
                0x0080014c                time_set
 .data          0x008001b7        0x0 spi1.o
 .data          0x008001b7        0x0 i2c.o
 .data          0x008001b7        0x0 c:/winavr-20100110/bin/../lib/gcc/avr/4.3.3/avr4\libgcc.a(_udivmodhi4.o)
 .data          0x008001b7        0x0 c:/winavr-20100110/bin/../lib/gcc/avr/4.3.3/avr4\libgcc.a(_exit.o)
 .data          0x008001b7        0x0 c:/winavr-20100110/bin/../lib/gcc/avr/4.3.3/avr4\libgcc.a(_copy_data.o)
 .data          0x008001b7        0x0 c:/winavr-20100110/bin/../lib/gcc/avr/4.3.3/avr4\libgcc.a(_clear_bss.o)
 .data          0x008001b7        0x0 c:/winavr-20100110/bin/../lib/gcc/avr/4.3.3/../../../../avr/lib/avr4\libc.a(strtok.o)
 .data          0x008001b7        0x0 c:/winavr-20100110/bin/../lib/gcc/avr/4.3.3/../../../../avr/lib/avr4\libc.a(memcmp.o)
 .data          0x008001b7        0x0 c:/winavr-20100110/bin/../lib/gcc/avr/4.3.3/../../../../avr/lib/avr4\libc.a(memset.o)
 .data          0x008001b7        0x0 c:/winavr-20100110/bin/../lib/gcc/avr/4.3.3/../../../../avr/lib/avr4\libc.a(strcpy.o)
 .data          0x008001b7        0x0 c:/winavr-20100110/bin/../lib/gcc/avr/4.3.3/../../../../avr/lib/avr4\libc.a(strstr.o)
 .data          0x008001b7        0x0 c:/winavr-20100110/bin/../lib/gcc/avr/4.3.3/../../../../avr/lib/avr4\libc.a(strtok_r.o)
 .data          0x008001b7        0x0 c:/winavr-20100110/bin/../lib/gcc/avr/4.3.3/../../../../avr/lib/avr4\libc.a(eerd_block_atmega88.o)
 .data          0x008001b7        0x0 c:/winavr-20100110/bin/../lib/gcc/avr/4.3.3/../../../../avr/lib/avr4\libc.a(eerd_byte_atmega88.o)
 .data          0x008001b7        0x0 c:/winavr-20100110/bin/../lib/gcc/avr/4.3.3/../../../../avr/lib/avr4\libc.a(eewr_block_atmega88.o)
 .data          0x008001b7        0x0 c:/winavr-20100110/bin/../lib/gcc/avr/4.3.3/../../../../avr/lib/avr4\libc.a(eewr_byte_atmega88.o)
 *(.data*)
 *(.rodata)
 *(.rodata*)
 *(.gnu.linkonce.d*)
                0x008001b8                . = ALIGN (0x2)
 *fill*         0x008001b7        0x1 00
                0x008001b8                _edata = .
                0x008001b8                PROVIDE (__data_end, .)

.bss            0x008001b8      0x14e
                0x008001b8                PROVIDE (__bss_start, .)
 *(.bss)
 .bss           0x008001b8        0x0 c:/winavr-20100110/bin/../lib/gcc/avr/4.3.3/../../../../avr/lib/avr4/crtm88.o
 .bss           0x008001b8        0x4 cc1100.o
 .bss           0x008001bc        0xd main.o
                0x008001c6                gRecvRssi
                0x008001bc                wakeup_condition
                0x008001c2                tampa_status
                0x008001bf                sr_status
                0x008001c7                gRecvLqi
                0x008001c4                setup_mode
                0x008001bd                get_user0_data
                0x008001c8                gStatus
                0x008001c1                emg_status
                0x008001c0                sr_status_old
                0x008001be                uart_rx_index
                0x008001c5                gslave_master_ctl
                0x008001c3                tampa_status_old
 .bss           0x008001c9        0x1 spi1.o
                0x008001c9                spi_active
 .bss           0x008001ca        0x1 i2c.o
                0x008001ca                i2c_error_flag
 .bss           0x008001cb        0x0 c:/winavr-20100110/bin/../lib/gcc/avr/4.3.3/avr4\libgcc.a(_udivmodhi4.o)
 .bss           0x008001cb        0x0 c:/winavr-20100110/bin/../lib/gcc/avr/4.3.3/avr4\libgcc.a(_exit.o)
 .bss           0x008001cb        0x0 c:/winavr-20100110/bin/../lib/gcc/avr/4.3.3/avr4\libgcc.a(_copy_data.o)
 .bss           0x008001cb        0x0 c:/winavr-20100110/bin/../lib/gcc/avr/4.3.3/avr4\libgcc.a(_clear_bss.o)
 .bss           0x008001cb        0x2 c:/winavr-20100110/bin/../lib/gcc/avr/4.3.3/../../../../avr/lib/avr4\libc.a(strtok.o)
 .bss           0x008001cd        0x0 c:/winavr-20100110/bin/../lib/gcc/avr/4.3.3/../../../../avr/lib/avr4\libc.a(memcmp.o)
 .bss           0x008001cd        0x0 c:/winavr-20100110/bin/../lib/gcc/avr/4.3.3/../../../../avr/lib/avr4\libc.a(memset.o)
 .bss           0x008001cd        0x0 c:/winavr-20100110/bin/../lib/gcc/avr/4.3.3/../../../../avr/lib/avr4\libc.a(strcpy.o)
 .bss           0x008001cd        0x0 c:/winavr-20100110/bin/../lib/gcc/avr/4.3.3/../../../../avr/lib/avr4\libc.a(strstr.o)
 .bss           0x008001cd        0x0 c:/winavr-20100110/bin/../lib/gcc/avr/4.3.3/../../../../avr/lib/avr4\libc.a(strtok_r.o)
 .bss           0x008001cd        0x0 c:/winavr-20100110/bin/../lib/gcc/avr/4.3.3/../../../../avr/lib/avr4\libc.a(eerd_block_atmega88.o)
 .bss           0x008001cd        0x0 c:/winavr-20100110/bin/../lib/gcc/avr/4.3.3/../../../../avr/lib/avr4\libc.a(eerd_byte_atmega88.o)
 .bss           0x008001cd        0x0 c:/winavr-20100110/bin/../lib/gcc/avr/4.3.3/../../../../avr/lib/avr4\libc.a(eewr_block_atmega88.o)
 .bss           0x008001cd        0x0 c:/winavr-20100110/bin/../lib/gcc/avr/4.3.3/../../../../avr/lib/avr4\libc.a(eewr_byte_atmega88.o)
 *(.bss*)
 *(COMMON)
 COMMON         0x008001cd      0x139 main.o
                0x008001cd                uart_rx_length
                0x008001ce                uart_data
                0x008001cf                gTestMode
                0x008001d0                SRBufIndex
                0x008001d1                gOpt
                0x008001e0                tSlave
                0x008001e4                pC
                0x008001e6                gClient
                0x0080022f                gLevel
                0x00800230                gggLength
                0x00800231                tSlave2
                0x00800235                gTemperature
                0x00800237                SRBuf
                0x0080023b                gWCmd
                0x0080029b                tCtl
                0x008002a2                rx_char
                0x008002de                cmd
                0x00800306                PROVIDE (__bss_end, .)
                0x00001db2                __data_load_start = LOADADDR (.data)
                0x00001e6a                __data_load_end = (__data_load_start + SIZEOF (.data))

.noinit         0x00800306        0x0
                0x00800306                PROVIDE (__noinit_start, .)
 *(.noinit*)
                0x00800306                PROVIDE (__noinit_end, .)
                0x00800306                _end = .
                0x00800306                PROVIDE (__heap_start, .)

.eeprom         0x00810000      0x1bc
 *(.eeprom*)
 .eeprom        0x00810000      0x1bc main.o
                0x008101b7                monitor_state
                0x008101ba                cnt_loop_break
                0x00810007                greg_slave
                0x008101b3                eprom_fixid
                0x00810197                eprom_level
                0x008101b8                wdt_cnt
                0x008101b6                test_mode
                0x00810000                gctl_data
                0x008101bc                __eeprom_end = .

.fuse
 *(.fuse)
 *(.lfuse)
 *(.hfuse)
 *(.efuse)

.lock
 *(.lock*)

.signature
 *(.signature*)

.stab
 *(.stab)

.stabstr
 *(.stabstr)

.stab.excl
 *(.stab.excl)

.stab.exclstr
 *(.stab.exclstr)

.stab.index
 *(.stab.index)

.stab.indexstr
 *(.stab.indexstr)

.comment
 *(.comment)

.debug
 *(.debug)

.line
 *(.line)

.debug_srcinfo
 *(.debug_srcinfo)

.debug_sfnames
 *(.debug_sfnames)

.debug_aranges  0x00000000       0x80
 *(.debug_aranges)
 .debug_aranges
                0x00000000       0x20 cc1100.o
 .debug_aranges
                0x00000020       0x20 main.o
 .debug_aranges
                0x00000040       0x20 spi1.o
 .debug_aranges
                0x00000060       0x20 i2c.o

.debug_pubnames
                0x00000000      0xa82
 *(.debug_pubnames)
 .debug_pubnames
                0x00000000      0x1a1 cc1100.o
 .debug_pubnames
                0x000001a1      0x701 main.o
 .debug_pubnames
                0x000008a2       0xf5 spi1.o
 .debug_pubnames
                0x00000997       0xeb i2c.o

.debug_info     0x00000000     0x251e
 *(.debug_info)
 .debug_info    0x00000000      0x3f9 cc1100.o
 .debug_info    0x000003f9     0x1c35 main.o
 .debug_info    0x0000202e      0x29c spi1.o
 .debug_info    0x000022ca      0x254 i2c.o
 *(.gnu.linkonce.wi.*)

.debug_abbrev   0x00000000      0x8e0
 *(.debug_abbrev)
 .debug_abbrev  0x00000000      0x193 cc1100.o
 .debug_abbrev  0x00000193      0x4a8 main.o
 .debug_abbrev  0x0000063b      0x186 spi1.o
 .debug_abbrev  0x000007c1      0x11f i2c.o

.debug_line     0x00000000     0x2371
 *(.debug_line)
 .debug_line    0x00000000      0x372 cc1100.o
 .debug_line    0x00000372     0x1ac4 main.o
 .debug_line    0x00001e36      0x26a spi1.o
 .debug_line    0x000020a0      0x2d1 i2c.o

.debug_frame    0x00000000      0x6a0
 *(.debug_frame)
 .debug_frame   0x00000000      0x110 cc1100.o
 .debug_frame   0x00000110      0x420 main.o
 .debug_frame   0x00000530       0xb0 spi1.o
 .debug_frame   0x000005e0       0xc0 i2c.o

.debug_str      0x00000000      0xc83
 *(.debug_str)
 .debug_str     0x00000000      0x25a cc1100.o
                                0x2ab (size before relaxing)
 .debug_str     0x0000025a      0x8a0 main.o
                                0xa52 (size before relaxing)
 .debug_str     0x00000afa       0xcc spi1.o
                                0x1e1 (size before relaxing)
 .debug_str     0x00000bc6       0xbd i2c.o
                                0x1a2 (size before relaxing)

.debug_loc      0x00000000      0xc8f
 *(.debug_loc)
 .debug_loc     0x00000000      0x182 cc1100.o
 .debug_loc     0x00000182      0x94e main.o
 .debug_loc     0x00000ad0       0xa7 spi1.o
 .debug_loc     0x00000b77      0x118 i2c.o

.debug_macinfo
 *(.debug_macinfo)
OUTPUT(CC1101driver.elf elf32-avr)
LOAD linker stubs

.debug_ranges   0x00000000       0xf0
 .debug_ranges  0x00000000       0xf0 main.o
